:100000008316BF3087002430980081309900831216
:10001000903098008317A03084008C1E0D2818198A
:100020001C28981821281A0880000D3C031926283E
:10003000840A031D0D2826281A083F308000981CCA
:100040001828181218163F3080001828A030840095
:100050000008482000080D3C03193228840A031DBB
:1000600028283228A10121083B20003E03190A2834
:100070004820A10A332882078F3449349734B93491
:1000800000340034003400340034003400340034D0
:10009000A0008316981C4A288312200899000800A3
:00000001FF
